:1000000012C0189518951895189518951895189563
:10001000C5C7C8C3189518951895189518951895BB
:100020001895189518958FE58DBFC8E3E0E24E2E20
:1000300084E08EBFD4E0F4E05F2EA89584B7082E4C
:10004000877F84BF88E1992781BD91BDEEEFF3E002
:10005000A0E6B0E088278D933197E9F76624A09851
:10006000A89AA198A99AA298AA9A8FEF81BB8FEF1C
:1000700087BBEAE1F0E0A4E9B0E091E0BBDE98994B
:1000800057C081E08093620000916200083C10F04C
:1000900009F04EC000916200063909F03CC0809121
:1000A0008E00806880938E00A4E9B0E08C9198E087
:1000B00089278C93EAE1F0E0A4E9B0E091E07BE7E6
:1000C00088DE00919400003009F00EC09298969856
:1000D000C798C2989098C6989798C598919A949AFC
:1000E000939AC19AC09A959A00919400083009F0A9
:1000F0000EC0929A969AC79AC29A909AC69A979A5E
:10010000C59A919894989398C198C09895988CEDB9
:1001100095E0F4DB0DC0989B01C00AC08AE090E036
:10012000EDDBA2E6B0E08C918F5F8C9308F4ACCF4E
:10013000E4E1F0E0A0E1B0E05ADE0F3F09F05AC080
:100140008EE591E0A7E7B0E08D939C938CE291E07F
:10015000A5E7B0E08D939C9388E191E0ADE7B0E036
:100160008D939C938AEF90E0ABE7B0E08D939C93E6
:1001700080E0809394008BEB809391008BEB8093D5
:100180009200E0E0F0E0A5E7B0E092E07BE721DE5E
:10019000E5E0F0E0A7E7B0E092E07BE71ADEEAE016
:1001A000F0E0ABE7B0E092E07BE713DEEEE0F0E0FA
:1001B000ADE7B0E092E07BE70CDEE0E1F0E0A1E942
:1001C000B0E091E07BE705DEE1E1F0E0A2E9B0E03C
:1001D00091E07BE7FEDDEAE1F0E0A4E9B0E091E048
:1001E0007BE7F7DDE4E1F0E0A0E1BB2784E68C9358
:1001F0007BE7ECDDE0E0F0E0A5E7B0E092E0FADDDF
:10020000E5E0F0E0A7E7B0E092E0F4DDEAE0F0E05E
:10021000ABE7B0E092E0EEDDEEE0F0E0ADE7B0E0BD
:1002200092E0E8DDE0E1F0E0A1E9B0E091E0E2DDBC
:10023000E1E1F0E0A2E9B0E091E0DCDD83E083BF42
:1002400080E08FBD81E08EBD789489B7816089BFE1
:1002500089B7846089BF83E083BF81E08EBD85E07C
:1002600080939B0080918E00886080938E008091A7
:100270008E00846080938E0080E190E0A5E6B0E07F
:100280008D939C9385E090E0A7E6B0E08D939C93DE
:1002900081E090E0A9E6B0E08D939C9380E190E04E
:1002A000ABE6B0E08D939C9385E090E0ADE6B0E0E6
:1002B0008D939C9382E090E0AFE6B0E08D939C93A9
:1002C00080ED97E01BDB80918E00877F80938E000E
:1002D00080918E008B7F80938E00AFEAB0E082B772
:1002E0008C93ADEAB0E08C9181FB81E00EF480E06C
:1002F0008F930091AF00023381E008F080E09F917E
:100300008923882309F421C0ABE9B0E08C91E3E3B1
:10031000EEDC81E08A93ABE9B0E08C916CECBB271A
:10032000A6E1E3E306DD81E08A93ABE9B0E08C91DE
:1003300064E4BB27A6E1E3E3FCDC8091AD008260CE
:100340008093AD0080E08093AE00AFEAB0E082B76A
:100350008C93ADEAB0E08C9182FB81E00EF080E0FE
:100360008F930091AF00023381E008F080E09F910D
:100370008923882309F443C1ABE9B0E08C91E3E31E
:10038000B6DC81E08A93ABE9B0E08C916CECBB27E2
:10039000A6E1E3E3CEDC81E08A93ABE9B0E08C91A7
:1003A0006EEBBB27A6E1E3E3C4DCABE9B0E08C91E4
:1003B000AEE9B0E0E3E329E02A93DADC88E0EEE995
:1003C000F0E01FDD402F0091A600041709F0F0C0F7
:1003D00080919E0080939C0080919F0080939D005F
:1003E00000919D00083F08F426C000E040919C0069
:1003F000041BACE9B0E00C930FEF40919D00041B8F
:10040000ADE9B0E00C9362FA0EF414C000919B00C9
:10041000053009F005C08091AD0080648093AD0087
:1004200000919B00043009F005C08091AD0080620E
:100430008093AD0014C000919B00053009F005C009
:100440008091AD008F7B8093AD0000919B000430C4
:1004500009F005C08091AD008F7D8093AD00E2E290
:10046000FEE1FFDBECE9F0E0D080EE24FF24002782
:10047000CADA15DBEDE0F0E0A7EAB0E09BDCADE91D
:10048000B0E00D91112740E150E047DAABEAB0E06F
:100490000D931C93EBEAF0E0D190E0808FEFE7FE44
:1004A0008827F82E082FAFDADFDAE7EAF0E087DAFC
:1004B00086DBEDE0F0E0A7EAB0E07CDCE6E2FEE11E
:1004C000D0DBE7EAF0E07BDA40DBEDE0F0E0A7EA42
:1004D000B0E070DC00919B00053009F005C0E7EA50
:1004E000F0E0A5E9B0E066DC00919B00043009F083
:1004F0000AC0E7EAF0E025DAA9E9B0E0EE0C000F67
:10050000E794DD92EC9262FA0EF452C0E5E9F0E075
:1005100056DAEAE2FEE1A5DBADDB10F009F001C03E
:1005200006C08091AD0080618093AD0005C08091D0
:10053000AD008F7E8093AD00A9E9B0E00D911C91D4
:10054000073E53E0150714F009F001C006C0809182
:10055000AD0088608093AD0005C08091AD00877FBD
:100560008093AD00E5E9F0E0ECD9A1E7B0E0EE0C56
:10057000000FE794DD92EC92A9E9B0E08D919C9197
:10058000A9E7B0E08D939C9300919B00053009F0A2
:1005900005C080918E00816080938E0000919B0049
:1005A000043009F005C08091AD0080688093AD00F3
:1005B0008091AD008B7F8093AD008091AD008D7FE9
:1005C0008093AD0080E08093AE00AEE8B0E08C9107
:1005D00081FB882780F9809580FBAEE8B0E08C91A4
:1005E00081F98C93AEE8B0E08C9181FB0EF004C0F1
:1005F00084E080939B0003C085E080939B00ADEA7C
:10060000B0E08C9186FB0EF44DC0A7E7B0E04D91B1
:100610005C91A5E7B0E00D911C910417150708F057
:1006200021C0A5E7B0E04D915C91A1E7B0E00D914C
:100630001C910417150714F009F003C081E08093A2
:100640007F00A7E7B0E04D915C91A1E7B0E00D918C
:100650001C91041715070CF001C003C080E08093C3
:100660007F0020C0A5E7B0E04D915C91A1E7B0E02C
:100670000D911C91041715070CF001C003C081E017
:1006800080937F00A7E7B0E04D915C91A1E7B0E0D7
:100690000D911C910417150714F009F003C080E0B8
:1006A00080937F0000917F00013081E009F080E0BD
:1006B0008F93AEE8B0E08C9180FB81E00EF080E09B
:1006C0009F918923882309F402C0C39A01C0C3986B
:1006D000ADEAB0E08C9185FB0EF44DC0ADE7B0E023
:1006E0004D915C91ABE7B0E00D911C91041715079B
:1006F00008F021C0ABE7B0E04D915C91A9E7B0E014
:100700000D911C910417150714F009F003C081E046
:1007100080938000ADE7B0E04D915C91A9E7B0E037
:100720000D911C91041715070CF001C003C080E067
:100730008093800020C0ABE7B0E04D915C91A9E7C9
:10074000B0E00D911C91041715070CF001C003C017
:1007500081E080938000ADE7B0E04D915C91A9E726
:10076000B0E00D911C910417150714F009F003C0B7
:1007700080E08093800000918000013081E009F0EA
:1007800080E08F93ADEAB0E08C9187FB81E00EF0C2
:1007900080E09F918923882309F402C0C49A01C094
:1007A000C4989BCD0F921F922F923F924F925F92CF
:1007B0007F92AF92BF920F931F932F933F934F93CC
:1007C0005F936F937F938F939F93AF93BF93CF93D9
:1007D000DF93EF93FF938FB78F93882783BF0091A9
:1007E0008D00003081E009F480E08F93AEE8B0E046
:1007F0008C9185FB81E00EF480E09F918923882312
:1008000009F403C0AFE8B0E023D8AFE8B0E00D9141
:100810001C9108355BE1150710F009F001C009C013
:1008200080E090E0AFE8B0E08D939C9380E080930F
:100830008D0000918D00003009F011C0A1E7B0E0FB
:100840008D919C91A7E8B0E08D939C93A9E7B0E0CF
:100850008D919C91A9E8B0E08D939C934FC001309D
:1008600009F011C0A5E7B0E08D919C91A7E8B0E038
:100870008D939C93A9E7B0E08D919C91A9E8B0E09D
:100880008D939C933BC0023009F011C0A7E7B0E004
:100890008D919C91A7E8B0E08D939C93A9E7B0E07F
:1008A0008D919C91A9E8B0E08D939C9327C0033073
:1008B00009F011C0A1E7B0E08D919C91A7E8B0E0EC
:1008C0008D939C93ABE7B0E08D919C91A9E8B0E04B
:1008D0008D939C9313C0043009F010C0A1E7B0E0E1
:1008E0008D919C91A7E8B0E08D939C93ADE7B0E02B
:1008F0008D919C91A9E8B0E08D939C93AEE8B0E017
:100900008C9183FB0EF4ABC0A7E8B0E08D919C9175
:10091000A1E8B0E08D939C93A1E8B0E08D919C910B
:10092000A5E8B0E08D939C9383E0809363004091B1
:10093000630001E0041710F009F025C0A1E8B0E061
:100940000D911C914AE050E096D7A3E6B0E0AD903F
:10095000BB24A3E6B0E0AA0CBB1CAA0DBB1D0D93E3
:100960001C93A1E8B0E00D911C914AE050E083D7C0
:10097000A1E8B0E04D935C93809163008150809337
:10098000630008F0D4CFA5E8B0E00D911C910436C7
:1009900050E015070CF401C006C08BE090E0A5E61E
:1009A000B0E08D939C93ADEAB0E08C9186FB81E042
:1009B0000EF080E08F9300918D00013081E009F40A
:1009C00080E09F9189238F9300918D00023081E018
:1009D00009F480E09F918923882309F412C082E101
:1009E00090E0A5E6B0E08D939C9381E190E0A7E6CE
:1009F000B0E08D939C938BE090E0A9E6B0E08D93FE
:100A00009C93ADEAB0E08C9184FB81E00EF080E035
:100A10008F9300918D00013081E009F480E09F9177
:100A200089238F9300918D00023081E009F480E0EA
:100A30009F918923882309F412C083E190E0A5E601
:100A4000B0E08D939C9384E190E0A7E6B0E08D93B5
:100A50009C938BE090E0A9E6B0E08D939C93AEE888
:100A6000B0E08C9182FB0EF4ABC0A9E8B0E08D91B0
:100A70009C91A3E8B0E08D939C93A3E8B0E08D91A6
:100A80009C91A5E8B0E08D939C9386E080936300F1
:100A90004091630004E0041710F009F025C0A3E8BA
:100AA000B0E00D911C914AE050E0E5D6A3E6B0E03D
:100AB000AD90BB24A3E6B0E0AA0CBB1CAA0DBB1DE5
:100AC0000D931C93A3E8B0E00D911C914AE050E017
:100AD000D2D6A3E8B0E04D935C938091630081503F
:100AE0008093630008F0D4CFA5E8B0E00D911C918D
:100AF000043650E015070CF401C006C08BE090E00E
:100B0000ABE6B0E08D939C93ADEAB0E08C9185FBB1
:100B100081E00EF080E08F9300918D00033081E042
:100B200009F480E09F9189238F9300918D00043018
:100B300081E009F480E09F918923882309F412C0A1
:100B400082E190E0ABE6B0E08D939C9381E190E090
:100B5000ADE6B0E08D939C938BE090E0AFE6B0E023
:100B60008D939C93ADEAB0E08C9183FB81E00EF015
:100B700080E08F9300918D00033081E009F480E0E4
:100B80009F9189238F9300918D00043081E009F4B7
:100B900080E09F918923882309F412C083E190E0CB
:100BA000ABE6B0E08D939C9384E190E0ADE6B0E0DD
:100BB0008D939C938BE090E0AFE6B0E08D939C9397
:100BC00000919400003009F007C091989498939890
:100BD000C198C098959806C0919A949A939AC19A90
:100BE000C09A959AA0E6B0E08C918F5F8C930091AB
:100BF0006000063010F009F001C003C081E080936E
:100C0000600090D1A4E6B0E08C9186FBA2E3B0E056
:100C10008C9182F98C9386D1A4E6B0E08C9185FB0F
:100C2000A2E3B0E08C9186F98C937CD1A4E6B0E08D
:100C30008C9184FBA8E3B0E08C9187F98C9372D1FE
:100C4000A4E6B0E08C9183FBA8E3B0E08C9182F93C
:100C50008C9368D1A4E6B0E08C9182FBA2E3B0E073
:100C60008C9180F98C935ED1A4E6B0E08C9181FBED
:100C7000A8E3B0E08C9186F98C9354D1A4E6B0E05F
:100C80008C9180FBA2E3B0E08C9187F98C9300916A
:100C90006000013009F02FC000919400003009F08D
:100CA00013C0919AAEE8B0E08C9183FB0EF40AC0B9
:100CB000A1E9B0E08C9181FBA8E3B0E08C9185F9CB
:100CC0008C9301C0C59A16C09198AEE8B0E08C91A3
:100CD00083FB0EF40EC0A1E9B0E08C9183FBA8E386
:100CE000B0E08C9185F98C9388B390E2892788BB1A
:100CF00001C0C598F9C0023009F02FC000919400DE
:100D0000003009F013C0949AAEE8B0E08C9183FBF8
:100D10000EF40AC0A1E9B0E08C9182FBA8E3B0E038
:100D20008C9185F98C9301C0C59A16C09498AEE851
:100D3000B0E08C9183FB0EF40EC0A1E9B0E08C9181
:100D400082FBA8E3B0E08C9185F98C9388B390E2A4
:100D5000892788BB01C0C598C7C0033009F02FC0E0
:100D600000919400003009F013C0939AAEE8B0E00F
:100D70008C9183FB0EF40AC0A1E9B0E08C9183FB57
:100D8000A8E3B0E08C9185F98C9301C0C59A16C098
:100D90009398AEE8B0E08C9183FB0EF40EC0A1E90D
:100DA000B0E08C9181FBA8E3B0E08C9185F98C9345
:100DB00088B390E2892788BB01C0C59895C00430EC
:100DC00009F02FC000919400003009F013C0C19ABF
:100DD000AEE8B0E08C9182FB0EF40AC0A2E9B0E06C
:100DE0008C9181FBA8E3B0E08C9185F98C9301C0D4
:100DF000C59A16C0C198AEE8B0E08C9182FB0EF4A3
:100E00000EC0A2E9B0E08C9183FBA8E3B0E08C9126
:100E100085F98C9388B390E2892788BB01C0C59877
:100E200063C0053009F02FC000919400003009F034
:100E300013C0C09AAEE8B0E08C9182FB0EF40AC0F9
:100E4000A2E9B0E08C9182FBA8E3B0E08C9185F937
:100E50008C9301C0C59A16C0C098AEE8B0E08C91E2
:100E600082FB0EF40EC0A2E9B0E08C9182FBA8E3F5
:100E7000B0E08C9185F98C9388B390E2892788BB88
:100E800001C0C59831C0063009F02EC00091940011
:100E9000003009F013C0959AAEE8B0E08C9182FB67
:100EA0000EF40AC0A2E9B0E08C9183FBA8E3B0E0A5
:100EB0008C9185F98C9301C0C59A16C09598AEE8BF
:100EC000B0E08C9182FB0EF40EC0A2E9B0E08C91F0
:100ED00081FBA8E3B0E08C9185F98C9388B390E214
:100EE000892788BB01C0C59883E083BF8F918FBFDE
:100EF000FF91EF91DF91CF91BF91AF919F918F9132
:100F00007F916F915F914F913F912F911F910F9121
:100F1000BF90AF907F905F904F903F902F901F9029
:100F20000F901895A0E6B0E0AD90BB24A3E6B0E02A
:100F3000AA0CBB1CAA0DBB1D8C9180936400009170
:100F40009400003009F00AC0E0E7FFE0A4E6B0E05A
:100F50008C919927A4E6B0E0AFD609C0E6E8FFE09F
:100F6000A4E6B0E08C919927A4E6B0E0A5D6089558
:100F7000014F12064C24200F00047E7F6A38307A1D
:100F800042E2F1C8FB007E306D79335B5F707F7B9E
:100F9000010015474F053D1D0E3704000F921F92AB
:100FA0002F923F924F925F927F92AF92BF920F9398
:100FB0001F932F933F934F935F936F937F938F93E1
:100FC0009F93AF93BF93CF93DF93EF93FF938FB72D
:100FD0008F93A2E6B0E08C918F5F8C93ADEAB0E086
:100FE0008C9181FB81E00EF080E08F930091AE0048
:100FF0000E3F81E008F080E09F918923882309F467
:1010000005C0AEEAB0E08C918F5F8C930091AE008A
:10101000043110F009F001C005C08091AD0084607A
:101020008093AD008EB5887F8EBDA3E3B0E00C91B8
:1010300000FB81E00EF480E08F93AEE8B0E08C918D
:1010400087FB81E00EF480E09F9189238F93A3E3D7
:10105000B0E00C9101FB81E00EF080E09F918923CC
:101060008F93A3E3B0E00C9102FB81E00EF080E0EF
:101070009F918923882309F401C0B7D0AEE8B0E07E
:101080008C9184FB81E00EF080E08F93A3E3B0E0CD
:101090000C9100FB81E00EF080E09F918923882372
:1010A00009F406C0999901C0E1D29A9901C03DD3D3
:1010B000A3E3B0E00C9100FB81E00EF480E08F939D
:1010C000A3E3B0E00C9101FB81E00EF480E09F917E
:1010D00089238F9300918D00003081E009F080E03A
:1010E0009F9189238F93AEE8B0E08C9186FB81E0DD
:1010F0000EF480E09F918923882309F401C07CD3FA
:10110000A3E3B0E00C9100FB81E00EF480E08F934C
:10111000A3E3B0E00C9102FB81E00EF480E09F912C
:1011200089238F9300918D00003081E009F080E0E9
:101130009F9189238F93AEE8B0E08C9186FB81E08C
:101140000EF480E09F918923882309F401C06AD3BB
:10115000A3E3B0E00C9100FB81E00EF080E08F9300
:10116000A3E3B0E00C9101FB81E00EF080E09F91E1
:1011700089238F93A3E3B0E00C9102FB81E00EF092
:1011800080E09F918923882309F408C080918E0014
:101190008F7780938E0084E68093B000989B05C083
:1011A00080918E008F7B80938E0081E08EBD83E0E6
:1011B00083BF8F918FBFFF91EF91DF91CF91BF914F
:1011C000AF919F918F917F916F915F914F913F91DF
:1011D0002F911F910F91BF90AF907F905F904F9094
:1011E0003F902F901F900F901895789489B7816049
:1011F00089BF83E083BF80918E00806180938E00E1
:1012000080918E00806880938E0080E090E0AFE84F
:10121000B0E08D939C93A7E7B0E04D915C91A5E77A
:10122000B0E00D911C910417150781E009F080E0F2
:101230008F93ADE7B0E04D915C91ABE7B0E00D91DD
:101240001C910417150781E009F080E09F91892B1C
:10125000882309F401C0FDD0ADE8B0E08C918F5F28
:101260008C9300918D00043010F009F001C003C090
:1012700080E080938D0000918D00003009F043C024
:1012800080918E00886080938E0080918E008460B3
:1012900080938E008AE090E0A5E6B0E08D939C9369
:1012A0008AE090E0A7E6B0E08D939C938AE090E01E
:1012B000A9E6B0E08D939C938AE090E0ABE6B0E0C5
:1012C0008D939C938AE090E0ADE6B0E08D939C9383
:1012D0008AE090E0AFE6B0E08D939C9380918E0021
:1012E0008F7E80938E0084EF91E008D38EB5887F47
:1012F0008EBD882783BFEEE0F0E0ADE7B0E092E07E
:101300007BE767D59BC0013009F01BC080918E0040
:10131000886080938E0081E090E0A9E6B0E08D9334
:101320009C938CE090E0A7E6B0E08D939C9380E0E6
:1013300090E0A5E6B0E08D939C9384EF91E0DED23F
:101340007DC0023009F027C080918E0088608093B4
:101350008E0081E090E0A9E6B0E08D939C938DE053
:1013600090E0A7E6B0E08D939C9380E090E0A5E646
:10137000B0E08D939C9384EF91E0C0D28EB5887FCE
:101380008EBD882783BFE0E0F0E0A5E7B0E092E003
:101390007BE71FD553C0033009F027C080918E0032
:1013A000846080938E0082E090E0AFE6B0E08D93A1
:1013B0009C938CE090E0ADE6B0E08D939C9380E050
:1013C00090E0ABE6B0E08D939C9384EF91E096D2F1
:1013D0008EB5887F8EBD882783BFE5E0F0E0A7E764
:1013E000B0E092E07BE7F5D429C0043009F026C0D4
:1013F00080918E00846080938E0082E090E0AFE662
:10140000B0E08D939C938DE090E0ADE6B0E08D93DD
:101410009C9380E090E0ABE6B0E08D939C9384EFEA
:1014200091E06CD28EB5887F8EBD882783BFEAE0BD
:10143000F0E0ABE7B0E092E07BE7CBD480918E00A8
:10144000877F80938E0080918E008B7F80938E00AB
:10145000089580918E00806280938E00A7E7B0E0AF
:101460004D915C91A5E7B0E00D911C910417150713
:1014700009F059C080918E00886080938E008FE0C3
:1014800090E0A5E6B0E08D939C9380E190E0A7E624
:10149000B0E08D939C9380E190E0A9E6B0E08D935D
:1014A0009C9384EF91E02AD28BE090E0A5E6B0E037
:1014B0008D939C938BE090E0A7E6B0E08D939C9396
:1014C0008BE090E0A9E6B0E08D939C9384EF91E0EF
:1014D00015D28FE090E0A5E6B0E08D939C9380E17B
:1014E00090E0A7E6B0E08D939C9380E190E0A9E6C0
:1014F000B0E08D939C9384EF91E000D28BE090E07C
:10150000A5E6B0E08D939C938BE090E0A7E6B0E079
:101510008D939C938BE090E0A9E6B0E08D939C9333
:1015200084EF91E0EBD1ADE7B0E04D915C91ABE79A
:10153000B0E00D911C910417150709F059C0809176
:101540008E00846080938E008FE090E0ABE6B0E088
:101550008D939C9380E190E0ADE6B0E08D939C93F9
:1015600080E190E0AFE6B0E08D939C9384EF91E052
:10157000C5D18BE090E0ABE6B0E08D939C938BE01F
:1015800090E0ADE6B0E08D939C938BE090E0AFE609
:10159000B0E08D939C9384EF91E0B0D18FE090E028
:1015A000ABE6B0E08D939C9380E190E0ADE6B0E0D7
:1015B0008D939C9380E190E0AFE6B0E08D939C9397
:1015C00084EF91E09BD18BE090E0ABE6B0E08D93AF
:1015D0009C938BE090E0ADE6B0E08D939C938BE024
:1015E00090E0AFE6B0E08D939C9384EF91E086D1DC
:1015F00000918D00003009F001C027C0013009F0D2
:1016000007C0E0E0F0E0A5E7B0E092E0F3D31DC052
:10161000023009F007C0E5E0F0E0A7E7B0E092E0B3
:10162000E9D313C0033009F007C0EAE0F0E0ABE70C
:10163000B0E092E0DFD309C0043009F006C0EEE06C
:10164000F0E0ADE7B0E092E0D5D380918D0081501D
:1016500080938D0080E090E0AFE8B0E08D939C93A4
:1016600080918E008F7D80938E000895789489B745
:10167000816089BF83E083BF80E090E0AFE8B0E0A5
:101680008D939C930091B0000A3010F009F001C0D6
:1016900005C0A0EBB0E08C9185508C9300918D003B
:1016A000013009F00DC0A5E7B0E00D911C91073E97
:1016B00053E0150708F003C0A5E7B0E0C9D02FC07C
:1016C000023009F00DC0A7E7B0E00D911C91073E74
:1016D00053E0150708F003C0A7E7B0E0B9D01FC07A
:1016E000033009F00DC0ABE7B0E00D911C91073E4F
:1016F00053E0150708F003C0ABE7B0E0A9D00FC076
:10170000043009F00CC0ADE7B0E00D911C91073E2C
:1017100053E0150708F003C0ADE7B0E099D0A0EBA7
:10172000B0E08C919927EAD00895789489B78160C8
:1017300089BF83E083BF80E090E0AFE8B0E08D93A5
:101740009C930091B0000A3010F009F001C005C070
:10175000A0EBB0E08C9185508C9300918D0001300E
:1017600009F00FC0A5E7B0E00D911C91003050E0EA
:10177000150710F009F001C003C0A5E7B0E06FD075
:1017800035C0023009F00FC0A7E7B0E00D911C9101
:10179000003050E0150710F009F001C003C0A7E7C2
:1017A000B0E05DD023C0033009F00FC0ABE7B0E07C
:1017B0000D911C91003050E0150710F009F001C0A8
:1017C00003C0ABE7B0E04BD011C0043009F00EC04D
:1017D000ADE7B0E00D911C91003050E0150710F01E
:1017E00009F001C003C0ADE7B0E039D0A0EBB0E034
:1017F0008C91992783D0089580918E008064809386
:101800008E0091E0A1E9B0E092D08EB5887F8EBDC8
:10181000882783BFE0E1F0E0A1E9B0E091E07BE759
:10182000D8D2089580918E00806480938E0091E0DC
:10183000A2E9B0E07CD08EB5887F8EBD882783BFBB
:10184000E1E1F0E0A2E9B0E091E07BE7C2D20895E7
:10185000ED91FC91EF5FFF4FFC93EE930895ED91B6
:10186000FC91E150F040FC93EE93089508D055D0E0
:1018700000FC10D0089503D01ED001F8F9CF002449
:10188000E89457FF02C009D0689400F80BD010F814
:101890000124089502D009D00895509540954F5FD6
:1018A0005F4F0895E89417FF0895009510950F5F16
:1018B0001F4F68940895352F242FE894452B11F479
:1018C00068940895512F402F0027112780E1440F7D
:1018D000551F001F111F021B130B416018F4020F4C
:1018E000131F4E7F8A9599F708953197F1F7089560
:1018F000689462F80895E89462F80895EF93FF936E
:10190000EE27E82BE92B31F0E0EDF7E03197F1F726
:101910000197D1F7FF91EF9108950F92B801469F7B
:101920008001479F100D569F100D0F900895903025
:1019300039F08C91880F08F481609A95D9F78C93CF
:1019400008953DD0992711278F2D880F80E8F82A18
:10195000802F881F08F41FEF41F08F57082F07FDD5
:1019600004C0003240F08FEF01C08827982FD82E96
:10197000E82EF82E09C08FE1801B082FF694E7941B
:10198000D79497950A95D1F7112351F09095D0945B
:10199000E094F09481E0980F8827D81EE81EF81E86
:1019A0000F2DFE2CED2CD92E0895D094E094F094B8
:1019B00091E0D90E9927E91EF91E10950895D1904E
:1019C000E190F190019108952191319141915191CE
:1019D0000895102F90E8FF0C001F0927990FF79426
:1019E0001078652F90E8440F551F5927990F479598
:1019F000607800380895FF0C90E89027110F9795B4
:101A0000F794092F0895102FBD2CDE2CEF2CF02E0B
:101A100011234AF4B094D094E094F0949FEFB91A53
:101A2000D90AE90AF90A0EE1FF2039F4FE2CED2C5F
:101A3000DB2CBB240850C2F766C032F00A95BB0C01
:101A4000DD1CEE1CFF1CF9CF01D0D5CFB7FE0895E9
:101A500090E8B91611F4D0FE08959FEFD91AE90A5B
:101A6000F90A09F403950895502F2D2D3E2D4F2D81
:101A7000612F08952DEC3CEC4CEC5DE366270FC024
:101A80009EDFF2DFDD24EE2490E8F92E0FE307C09D
:101A90009BDF05C02227332740E251E46627552308
:101AA00051F1002381F195DF71F11627005850584C
:101AB0000894050B18F407FD03C025C007FD23C0DB
:101AC000469537952795F694E794D79422D0FF2032
:101AD0002AF0DD0CEE1CFF1C015073F09D2D969535
:101AE00048F0DD203AF4EE202AF491E0D90E99274F
:101AF000E91EF91E80CF07C09FE7092FF92A9FEF43
:101B0000D92EE92E0895DD24EE24FF240027112785
:101B100008959F929924AA24BB2488E1D216E30653
:101B2000F40628F0D21AE30AF40A089401C0889453
:101B3000991CAA1CBB1CDD0CEE1CFF1C8A9571F7BE
:101B4000D92CEA2CFB2C9F90089543DFE1F250380A
:101B5000D1F21627005850580894051F12F418F4B3
:101B6000CBCF08F0D0CF0BD0FF202AF0BB0CDD1C70
:101B7000EE1CFF1C40CF0F5F0BF4BECF3CCF9F92FB
:101B80009924AA24BB24992788E1990CAA1CBB1C80
:101B9000DD1CEE1CFF1C30F4920EA31EB41ED91ED9
:101BA000E91EF91E8A9589F79F9008950AF045D09D
:101BB00022CF5FE322273327442701C005DF09DF57
:101BC0005038B1F3003899F3902F951B8BF312F432
:101BD00034D0FACF983118F0222733274427983091
:101BE00028F0232F342F44279850F9CF992329F038
:101BF0004695379527959A95D9F7912F962742F0D4
:101C000014D0B0F6F794E794D7940F5F8BF674CFA7
:101C100010D051F008F4C9DEFF2052F2DD0CEE1CAA
:101C2000FF1C0150CBF768CF6ECFD20EE31EF41E1F
:101C30000895D21AE30AF40A0895DF92EF92FF9210
:101C40000F931F93D22EE32EF42E052F162F6F9194
:101C50005F914F913F912F910895C8953196002043
:101C60000895FBDF202DF9DF302DF7DF402DF5DF64
:101C7000502D089507FB00680EF40F7757FB50684E
:101C80000EF45F7707FD02C057FF05C0D216E306CA
:101C9000F406050708952D153E054F0550070895D4
:101CA00091E005C092E003C094E001C098E0D5DF68
:101CB0000D929A95E1F70895E80FF91FF1CF91E0A1
:101CC000882321F08894991F8A95E9F7892F9095A8
:101CD00008950181082B0183128119231283EF9348
:101CE000FF93E8E0F0E001DEFF91EF91089503DE5D
:101CF000FF27E5DFEEDFEF93FF93ECEBF3E0F5DD9D
:101D0000FF91EF91182B128309230183EF93FF9327
:101D1000E8E8F0E0EADDFF91EF911081182309F087
:101D2000E7DDEF93FF93E0E3F3E0DFDDFF91EF9179
:101D30000895C5DFFF2729915D9148E0CADF5795D7
:101D400010F4182B1283EF93FF93E8E6F0E0CDDD5B
:101D5000FF91EF91182B1283EF93FF93E0E1F0E0F6
:101D6000C4DDFF91EF914A9549F72A9529F7089527
:101D7000A6DFFF27299148E05527ABDF0923018320
:101D8000EF93FF93EEE0F0E0B0DDFF91EF918894E8
:101D90001081182309F008945795EF93FF93EAE612
:101DA000F0E0A3DDFF91EF914A9539F75D932A9515
:101DB00011F7089594E081918D939A95E1F7089534
:101DC000E199FECFEEBBFFBB3196089591E001C0D3
:101DD00092E07B3751F47FB7F894F2DF8D918DBBA1
:101DE000E29AE19A9A95C9F77FBF7727089591E023
:101DF00001C092E0E5DFE09A8DB38D939A95D1F71B
:101E0000089500276CE8719198E00695779577FF23
:101E100018F477FD08F006279A95B9F78A9599F78F
:0E1E20000895000080410000204100C0794478
:00000001FF
